:020000040000FA
:0400000006303A2864
:08000800A000030EA100831209
:1000100005191028831601178312B23081002B288E
:1000200083160113831203140B190310A80DA90DD5
:10003000AA0DAB0DAC0DAC16FF302C02031D2B2806
:10004000FA302B02031D2B2831152A08AF0029088E
:10005000AE002808AD008B100B11210E8300A00EFE
:04006000200E090065
:0C007400203084008001840A6030040207
:10008000031C3C281230B00093218316FF239000FC
:10009000831283160C308505870183128501870141
:1000A000073099000030831691009F008312C830FA
:1000B00083168100831231309000003083168C004B
:1000C000831210308B00831600309B001C141A081A
:1000D0008312BC00831610309B001C141A08831274
:1000E000BD00E42181018E018F010B118B100B10DB
:1000F0008C018B17892031198C20B30B87280310B2
:1001000085190314B90DF030390203190821F521BE
:100110007A2864003210080031110130B7008B13C7
:100120002030370783169B001C141A088312A40082
:100130001030370783169B001C141A088312A30083
:10014000A6000230A6060030370783169B001C1459
:100150001A088312A200A7000130A7068B17321CD1
:10016000B72822090339A200A309A409A509240874
:100170002F02031D022923082E02031D0229220833
:100180002D02031D022901303702031DCC283D1822
:10019000CC283D143E149A2102303702031DD52885
:1001A000BD18D528BD143E14A12103303702031D0C
:1001B000DE283D19DE283D153E14A8210430370203
:1001C000031DE728BD19E728BD153E14AF210530F2
:1001D0003702031DF0283D1AF0283D163E14B621C3
:1001E00006303702031DF928BD1AF928BD163E1442
:1001F000BD2107303702031D02293D1B02293D178F
:100200003E14C421B70A08303702031808008F28AB
:100210000130B600B300B400B500B7008501870116
:10022000B1138920B30B4629031085190314B90DA6
:10023000F030390203196D29B40B46290130370219
:100240000319CC21023037020319CF2103303702C2
:100250000319D221043037020319D52105303702A2
:100260000319D821063037020319DB210730370282
:100270000319DE219630B4000330370232300319FF
:10028000B4000430370232300319B400311D112993
:100290003111321C50292D090339AD00AE09AF09C7
:1002A0002F1C11298E018F010C1C11290C102E1EE0
:1002B00011298B1320303707BB002F08BA0080218B
:1002C00010303707BB002E08BA00802100303707F6
:1002D000BB002D08BA0080218B1785018701B70A62
:1002E000B60108303702031C1129E42108003E1C26
:1002F00008003E101030BB003D08BA008021080005
:100300008B133A0883161C159A003B089B00553046
:100310009D00AA309D009C1464009C188C291C111F
:1003200083128B170800FF30D000D415D515D615D1
:10033000D7150800BD103D11BD110230CE00D2000E
:1003400008003D103D11BD110130CE00D200080063
:100350003D10BD10BD118230CE00D20008003D100E
:10036000BD103D114130CE00D2000800BD123D133A
:10037000BD130030CF00D30008003D123D13BD1364
:100380000230CF00D30008003D12BD12BD13013072
:10039000CF00D300080008000130850608000230B5
:1003A0008506080001308506080002308506080031
:1003B000303085060800103085060800203085069C
:1003C00008002230850608003D189A21BD18A12199
:1003D0003D19A821BD19AF213D1AB621BD1ABD2175
:1003E0003D1BC421BD1BCB2108008F080319080049
:1003F0008F0196308E00D00FAF2AD00ABD1A272A5F
:10040000521C272A521F182AD41C092AD401541519
:10041000352A541D0E2AD401D415352AD41D132A89
:10042000D4015416352A541E352AD401D414352A41
:10043000541D1D2AD4015416352AD41D222AD40154
:100440005416352A541E352AD401D414352AD41C06
:100450002C2AD4015415352A541D312AD401D4151F
:10046000352A541E352AD4015415BD1A5E2AD21CD1
:100470005E2AD21F4F2AD51C402AD50155156C2A59
:10048000551D452AD501D5156C2AD51D4A2AD501F9
:1004900055166C2A551E6C2AD501D5146C2A551D8B
:1004A000542AD50155166C2AD51D592AD501551641
:1004B0006C2A551E6C2AD501D5146C2AD51C632ACA
:1004C000D50155156C2A551D682AD501D5156C2AFC
:1004D000551E6C2AD5015515531C7D2A561D732AAD
:1004E000D60156168B2AD61D782AD60156168B2A87
:1004F000561E8B2AD601D6148B2AD61C822AD601E8
:1005000056158B2A561D872AD601D6158B2A561EBC
:100510008B2AD6015615D31C9C2A571D922AD70127
:100520005716AA2AD71D972AD7015716AA2A571E47
:10053000AA2AD701D714AA2AD71CA12AD70157154E
:10054000AA2A571DA62AD701D715AA2A571EAA2AB2
:10055000D701571577214E08D2004F08D300500815
:10056000D1000C305405031D85100C305505031DBA
:1005700005100C305605031D85120C305705031D60
:10058000051251080E020318D92A12305405031D12
:10059000851412305505031D051412305605031D30
:1005A000851612305705031D0516FF30500203193A
:1005B00008008F08031D0800892051080E02031C43
:1005C000D92A18305405031D851006305405031D23
:1005D000851418305505031D051006305505031DFB
:1005E000051418305605031D851206305605031DE7
:1005F000851618305705031D051206305705031DD3
:0406000005160800D3
:084000000E000300030008009C
:02400E00CC01E3
:10420000010078007A007C007E007B0079007F004E
:104210007D007A0078007E007C00FF00FF00FF0038
:104220000000F200F600FA00FE00F200F600FA00CC
:10423000FE00F200F600FA00FE00FF00FF00FF00A3
:10424000010005000500050005000900090009003E
:1042500009000D000D000D000D00FF00FF00FF0024
:10426000FF00FF00FF00FF00FF00FF00FF00FF0056
:10427000FF00FF00FF00FF00FF00FF00FF00FF0046
:10428000FF00FF00FF00FF00FF00FF00FF00FF0036
:10429000FF00FF00FF00FF00FF00FF00FF00FF0026
:1042A000FF00FF00FF00FF00FF00FF00FF00FF0016
:1042B000FF00FF00FF00FF00FF00FF00FF00FF0006
:1042C000FF00FF00FF00FF00FF00FF00FF00FF00F6
:1042D000FF00FF00FF00FF00FF00FF00FF00FF00E6
:1042E000FF00FF00FF00FF00FF00FF00FF00FF00D6
:1042F000FF00FF00FF00FF00FF00FF00FF00DD00E8
:00000001FF
